:020000040000FA
:0200000057D0D7
:0400080061EF19F09B
:08001800BCEF19F00F0B7C6E28
:10002000000EF76E360EF66E7C50F626D8B0F72A24
:100030000800F55012003031323334353637383954
:100040004142434445460F501F0B7C6E000EF76E35
:10005000540EE9D72C36404A545E68727C86909ADA
:10006000A4AEBECEDEEE070B7C6E000EF76E720EF7
:10007000DAD70A0E12161A1E59507C6ED8907C32AE
:100080007C327C301F0B7C6E000EF76E900ECBD74F
:1000900085786D645C56504B47433F3C393734326A
:1000A000302E2C2B292827262423222120201F1EF6
:1000B00029DB828AC5EC17F061DA2E8C72682D80FC
:1000C000010E526E100E8F6FFF0E056E06EC0CF0D7
:1000D0000650650810E121DA28E363DB010E365C87
:1000E00006E1B0EC0BF049DB58DBD4EF16F059DB3E
:1000F000040E365C16E1DFDA000EF86E380EF76E8D
:100100003A0EF66E73EC03F0DEEC0BF0D4DA000E70
:10011000F86E380EF76E4C0EF66E73EC03F00ADADA
:1001200023DAFBD9FEE258EF00F0000EF86E370E2E
:10013000F76EB60EF66E73EC03F05A6A056A06ECBB
:100140000CF0F1EC0BF0052A5A2EF9D79CEC02F0DA
:10015000B0EC0BF012DB0CDA0FC030F06FEC0BF0F0
:1001600010BC04D0FCEC08F01DEC09F051EC19F0C7
:1001700059EC19F051EC19F059EC19F01CEC0CF099
:1001800010B4838410B28384010E0E6E10A603D0C7
:100190002CB001D00E6A01DB726883B202D083B04A
:1001A00096D92E8837523CE010B483842E98F5DA25
:1001B00037502DA21ED037BE0BD07C0B31E0522A17
:1001C000050E10BC0D0E525C02E1010E526E0DD0F8
:1001D00037C05DF05D6C5D50FC0B22E0520652288A
:1001E00004E1040E10BC0C0E526E2E8C7268376A3D
:1001F00017D037BE09D0376A7F0B5D6E2EAA51EC3F
:1002000005F05D2EFBD709D0376C3750376A5D6E2D
:100210002EAA90EC05F05D2EFBD72E8C72682D80F7
:100220002EAC19EF01F02E9855EC07F026EC07F0F4
:100230002E9C2DA004D02E98CBDA2DDB2D906DD9DD
:100240002DAC20D010B483842E98A7DA2DA405D02D
:100250002D948DEC02F0FDE215D0A3DA010E365C90
:1002600002E1F7EC09F0020E365C02E105EC0AF05F
:10027000030E365C02E140EC0AF0040E365C02E14B
:100280007BEC0AF02FA003D02E982E8C72682F9A48
:10029000010E315C05E0020E315C02E02F8A1ED0B7
:1002A00010A81CD081B408D02DA205D02D84F9EC63
:1002B00017F02D9401D02E8281A22E842EA21CD064
:1002C0002E98EBDA83802D8483827CEC02F083927B
:1002D000F7D82D947CEC02F02E92F1D081B40AD0A4
:1002E00083B206D02E98D9DA838083822FAA2D84F8
:1002F000E7D8E5D083922D94010E315C03E0020E25
:10030000315C17E110A815D02EA413D02E98C5DAB1
:1003100083802D8483827CEC02F07CEC02F07CEC08
:1003200002F08392CDD8D3D82D947CEC02F02E9499
:10033000C6D0535209E02DAE12D010B283842D9E48
:100340002E802E8C72680AD02EA009D010B483940F
:1003500010B283842F902E902E8C72682E982CA031
:100360001DD057661BD0030E0E6E100ED06102D04A
:10037000020E0E6E0A0ED06102D0010E0E6E040E39
:10038000D06102D0000E0E6ED151D05D04E0D0C01D
:10039000D1F02E8C7268D06B0A0E576E2EA88FD0BB
:1003A000010E8F5D27E110ACFCEC08F00F50305CC3
:1003B00021E010ACDDD87FD930508ED9000EF86E18
:1003C000380EF76E060EF66E73EC03F089EC0BF048
:1003D00030C00FF06FEC0BF0ADD82E8C72682D8012
:1003E000DCD910B483842CB002D0010E0E6E10BC88
:1003F00051EC19F0020E8F5D1AE110AC1DEC09F002
:100400000F5201E1326A3250315C11E032C031F0FA
:100410002EA604D031C025F031C026F048EC0BF0F8
:10042000BCD910B483842D8010BC59EC19F0030E94
:100430008F5D08E110A006D02AEC08F06F50725CC6
:1004400001E02E8C040E8F5D23E110A821D07736B9
:10045000783677367836773678367736783678C0A5
:1004600075F05850785E10E075C078F05828785EC6
:100470000BE075C078F05804785E06E010B4838411
:100480002F808BD975C058F0756A766A776A786A5A
:10049000050E8F5D02E1CCEC17F0060E8F5D00E1DA
:1004A00010A809D03EEC09F08EC075F0766A755040
:1004B0007726765078228F2F02D0100E8F6F6DD650
:1004C000000ECE6EA60ECF6E12C054F01200010EBA
:1004D000315C04E0020E315C01E001D02D945452F5
:1004E00002E18390D8D912009EAAFED7AE50120026
:1004F0009EA8FED7AD6E12003EEC09F0BDDD566E33
:10050000F20ECB6ECA8481A42E8281A22E8483A295
:10051000DEDF5652F8E1CA9412002D9C8150F00B98
:10052000F00A03E02D8CD88001D0D890120001D8B9
:1005300001D800D802D801D800D8FA0E09D0C80EC8
:1005400007D0640E05D0320E03D00A0E01D0010E82
:10055000356E070E346E7D0E336E332EFED7342E7D
:10056000FCD7352EF6D712002D84EDDF2D94EBDF6E
:100570002D84E9DF2D9483908392120083968296D6
:100580008298E1DF200E78D8800E76D8DEDF200E4C
:1005900073D8800E71D8DBDF060E64D80C0E62D8DB
:1005A000140E60D830D887D8000EF86E330EF76E70
:1005B0008E0EF66E73EC03F0000EF86E330EF76ECF
:1005C000A00EF66E73EC03F0B4DF75D883841200CE
:1005D000076E5ED80750828682988396F00B4CD8BF
:1005E0000738F00B49D0076E07460746074650D834
:1005F0000750400937D8080E5A6E0900F550E8DF59
:100600005A2EFBD71200000EF86E060EF76E240E5F
:10061000F66E080E5B6E5C6A5C50E5DF5C2A5B2E52
:10062000FBD7120000001818181B000000001B1B4D
:100630001B1B000004041818181B040404041B1BD3
:100640001B1B0404001010101010100000141414D0
:100650001414140000000000001B00000404040433
:10066000041B0404076E14D80750F00B829682987E
:10067000839602D80738F00B83B0010983B20209D0
:1006800083B4040983B60809836E838683961200B7
:10069000838E958E829682882D968386000083AE07
:1006A0002D86839600008386000083962DA6F4D7BE
:1006B000959E82981200010ED5D7020ED3D7800ED8
:1006C000D1D7C00ECFD78009CDD7200E81D75A6E93
:1006D000FCDF5A2EFDD71200086E08389FDC78DF49
:1006E00008509CDC75D70900F550EDDF0900F55086
:1006F00002E06EDFFBD712000900F55002E0F8DEE1
:10070000FBD71200070EC16E860EC06E2F0E926EC2
:10071000FF0E936E800E946E000E956E070E966E11
:10072000000ED06EF00EF26E000EF16E000EF06E46
:10073000230E9D6E020EA06E010ECD6E210ECA6EAE
:10074000000EB16E2F0E806EFF0E816E270E826E30
:10075000000E836E070E846EFF0E5A6E00EE00F0E0
:10076000EE6A5A2EFDD710B4838410B28384000E33
:10077000CE6EA60ECF6ECDEF03F091D81C0E436E59
:10078000200E426EBFC04AF088DA58DA38C066F0F0
:10079000660ED66EC40ED56E1200C80E536E2D8E28
:1007A0001200280E5A6E8150F00B5B6ED0DE815025
:1007B000F00B5B5CF6E15A2EF6D7000E5BAE010E35
:1007C0005BAC020E5BAA030E5BA8040E366E120031
:1007D00066D89CD810EE42F0050E5A6EEE50E66ECA
:1007E0005A2EFCD70F5207E010A6FCEC04F02FA203
:1007F000E2D810BE44D809C04AF00AC04BF00BC082
:100800004CF00CC04DF00DC04EF0DED93CC05EF097
:100810003DC05FF03EC060F03FC061F040D87CD882
:1008200010EE42F0050E5A6EEE50E66E5A2EFCD7D0
:100830000F5211E010A6FCEC04F02FB20AD0010E0A
:10084000315C05E0020E315C02E094D802D010BAAF
:1008500091D810BE14D809C04AF00AC04BF00BC0A2
:100860004CF00CC04DF00DC04EF0AED93CC062F063
:100870003DC063F03EC064F03FC065F01200D89008
:10088000423643364436453646364236433644369B
:100890004536463612007DEF0CF08FEF0CF013D882
:1008A00009D8426A436A446A456A466A476A486A9E
:1008B000496A12004A6A4B6A4C6A4D6A4E6A4F6A2C
:1008C000506A516A1200386A396A3A6A3B6A3C6A6D
:1008D0003D6A3E6A3F6A406A416A120038C042F08F
:1008E00039C043F03AC044F03BC045F03CC046F04C
:1008F000120038C04AF039C04BF03AC04CF03BC04F
:100900004DF03CC04EF0120010EE38F000EE1BF03F
:100910002DB800EE20F012002EA6F8D700EE1BF046
:100920002DA800EE20F01200B1D8EECF38F0EECFB7
:1009300039F0EECF3AF0EECF3BF0200E5B6ED89060
:100940003B323A32393238323F323E323D323C323B
:1009500000EE38F0040E5A6EEFAE02D0300EEF5EAD
:10096000EFA602D0030EEF5EEE525A2EF5D75B2EA5
:10097000E6D712002FB409D0175042261850432250
:10098000195044221A50452208D01750425E185080
:10099000435A1950445A1A50455A45AE1200421E45
:1009A000431E441E451E422AD8B4432AD8B4442AC2
:1009B000D8B4452A12002FB409D01350422614503F
:1009C0004322155044221650452208D01350425E4F
:1009D0001450435A1550445A1650455A45AE120009
:1009E000421E431E441E451E422AD8B4432AD8B490
:1009F000442AD8B4452A1200466A5AEC04F00A0E7A
:100A00004A6E4DEC06F06EEC04F05AEC04F00A0E5F
:100A10004A6EE4EC05F06EEF04F009C042F00AC043
:100A200043F00BC044F00CC045F00DC046F0200E62
:100A30005B6E00EE42F010EE4AF0396AD8903F3219
:100A40003E323D323C32D8A015D0080E5A6E00EE30
:100A500042F010EE4AF0EECF38F03950396AE7260E
:100A600002E3010E396E3850E62602E3010E396EBC
:100A70005A2EF1D7D890423643364436453646365C
:100A80004736483649365B2ED4D71200416A406A51
:100A90003F6A3E6A3D6A3C6A3B6A3A6A396A386A2A
:100AA0001200F9DF31DF2CB00FD00E5031E0010E13
:100AB0000E5C2BE0020E0E5C25E0030E0E5C1AE0CD
:100AC000040E0E5C10E012000E5027E0010E0E5CCA
:100AD0001CE0020E0E5C16E0030E0E5C10E0040E2D
:100AE0000E5C01E01200A00E386E860E396E010E0B
:100AF0003A6E61D0030E396EE80E386E5CD0C80EC7
:100B0000386E59D0320E386E56D00A0E386E53D029
:100B1000382A51D0020E386E4ED0050E386E4BD0AA
:100B2000BADFF2DE2CB00FD00E5037E0010E0E5CB3
:100B30002BE0020E0E5C25E0030E0E5C1AE0040EA4
:100B40000E5C10E012000E5022E0010E0E5C1CE064
:100B5000020E0E5C16E0030E0E5C10E0040E0E5C3E
:100B600001E01200A00E386E860E396E010E3A6E4C
:100B700016D0030E396EE80E386E11D0C80E386EDE
:100B80000ED0320E386E0BD00A0E386E08D0050E1D
:100B9000386E05D0020E386E02D0382A00D0050E0D
:100BA0005A6ED86AE750D8A0E73CEF5EEE52E652A4
:100BB0005A2EF8D71200E650EE26040E5A6EE65072
:100BC000EE225A2EFCD712000A0E5A6E00EE38F0B2
:100BD000EE6A5A2EFDD72F9646BE40D84EBE4DD84F
:100BE000050E5A6E00EE4AF020EE38F0050E5B6EF0
:100BF0005A505B5E10EE42F020EE38F05B5203E09C
:100C0000DE525B2EFDD7050E5B6E030E5C6EEF5061
:100C1000E602F350DE26F450DE22E86ADE225C2E85
:100C2000FCD7040E5C6EDD525C2EFDD75B2EEDD73B
:100C3000EE525A2EDBD72FB601D81200381E391EBD
:100C40003A1E3B1E3C1E382AD8B4392AD8B43A2A58
:100C5000D8B43B2AD8B43C2A2F961200421E431E19
:100C6000441E451E461E422AD8B4432AD8B4442AFC
:100C7000D8B4452AD8B4462A0ED04A1E4B1E4C1E64
:100C80004D1E4E1E4A2AD8B44B2AD8B44C2AD8B48A
:100C90004D2AD8B44E2A2F7612002F9646BEDEDF9C
:100CA0004EBEEBDF4E9E469E5A6A0DDE5A2AD89003
:100CB0004EBE1BD04A364B364C364D364E364E5015
:100CC000465C0BE14D50455C08E14C50445C05E14D
:100CD0004B50435C02E14A50425CE8E2F4DDD890BC
:100CE0004E324D324C324B324A324E50465C0BE162
:100CF0004D50455C08E14C50445C05E14B50435C71
:100D000002E14A50425C0AE34A50425E4B50435A69
:100D10004C50445A4D50455A4E50465A3836393642
:100D20003A363B363C365A2EDAD72FB687DF1200DA
:100D3000386A396A3A6A3B6A3C6A3D6A280E5A6EDA
:100D4000060E5B6E00EE38F0EF500F0B7D6E050E59
:100D50007D5CD8A002D0030EEF26EF50F00B7D6E25
:100D6000500E7D5CD8A002D0300EEF26EC525B2EE8
:100D7000EBD7D89042364336443645364636383679
:100D800039363A363B363C363D365A2ED9D71200E4
:100D90002F9C8CBF2F8C8C9F00EE7EF00C0E5A6E19
:100DA0008A515A5C8A6F8B515A5C8B6F2D9A8C5189
:100DB0005A5E8B07D8B42D8A8B2B8B5303E12C0EF4
:100DC000E8EC02F0EE505B6E8A530CE12DBA06D0CF
:100DD000300E5B5C03E1200E5B6E01D02D8A5B5010
:100DE000E8EC02F08A5301E08A078B075A2EE1D71C
:100DF0008C5303E08C512FAC6ADC12007E6A7F6A50
:100E0000806B816B826B836B846B856B866B876B6E
:100E1000886B896B00EE7EF010EE3DF0060E5A6E88
:100E2000E7380F0B05D8E55003D85A2EF9D7120032
:100E30000F0B3009EE6E12000F0B04E12DAA02D049
:100E4000200E02D030092D9AE8EF02F02DB24AD2DE
:100E50002FB0CCD00F5202E010B044D1400E33DCA2
:100E6000410E2DA8420E2EA603D0610E2DA8620EB3
:100E7000E8EC02F02DB80BD020C042F021C043F0C6
:100E800022C044F023C045F024C046F00AD01BC065
:100E900042F01CC043F01DC044F01EC045F01FC00E
:100EA00046F032D8030E67EF03F0E86A63EC03F014
:100EB000410E2DB8420E2EA603D0610E2DB8620E43
:100EC000E8EC02F02DB80BD01BC042F01CC043F080
:100ED0001DC044F01EC045F01FC046F00AD020C01F
:100EE00042F021C043F022C044F023C045F024C0AA
:100EF00046F00AD82CA006D00C0E63EC03F02E0EA0
:100F0000E8EC02F09DEF07F000EE42F010EE27F063
:100F100052DE0EDF73DF0B0E8A6F060E8B6F010E33
:100F20008C6F2CB007D00EC08CF0040E0E5C02E16A
:100F3000050E8C6FC8EC06F012000D0E63EC03F08A
:100F400010BE02D0315209E1000EF86E370EF76E76
:100F5000DC0EF66E73EC03F01200010E315C09E159
:100F6000000EF86E370EF76EE20EF66E73EC03F0BD
:100F70001200020E315C09E1000EF86E370EF76EBA
:100F8000E80EF66E73EC03F01200030E315C09E11B
:100F9000000EF86E370EF76EEE0EF66E73EC03F081
:100FA0001200040E315C09E1000EF86E370EF76E88
:100FB000F40EF66E73EC03F01200050E315C09E1DD
:100FC000000EF86E370EF76EFA0EF66E73EC03F045
:100FD0001200060E315C09E1000EF86E380EF76E55
:100FE000000EF66E73EC03F0120012000F52D8B42C
:100FF0001200000EF86E380EF76E200EF66E73ECCF
:1010000003F03EEC09F05D6E5D325D325D301F0B2A
:10101000090F5D6E44DC5DC042F08ADE38506CEC36
:1010200003F0090E67EF03F0B7C04AF0B8C04BF009
:10103000B9C04CF0BAC04DF0BABF4E681200BBC088
:101040004AF0BCC04BF0BDC04CF0BEC04DF0BEBFBE
:101050004E6812004FEC04F04DEC09F08DC042F0E8
:101060008EC043F014EC08F0E4EC05F06EEC04F0F4
:101070001FEC08F04A5042264B5043224C50442269
:101080004D5045224E50462246BE51EC04F05AECDB
:1010900004F0500E4A6EC30E4B6E000E4C6E4A505A
:1010A00042264B5043224C5044224D5045224E5034
:1010B00046225AEC04F0A00E4A6E860E4B6E010ECC
:1010C0004C6E4DEC06F038C06FF038C071F0712AEC
:1010D000D890713242C070F06FAE03D06F6A706A00
:1010E000716A120072506F5CD8B448D06FC072F051
:1010F000400E63EC03F00D0E5A6E050E5A6202D0DC
:10110000070E01D0060EE8EC02F05A2EF6D7400E7C
:1011100063EC03F06FC05AF0D8905A325B6A5A52AF
:101120000EE05B2A0E0E5B6018D0090E5B6202D0E7
:10113000030E01D0010EE8EC02F05A2EF2D76FA098
:101140000CD05B2A0E0E5B6008D0090E5B6202D0E9
:10115000020E01D0000EE8EC02F04E0E63EC03F03C
:10116000530EE8EC02F0090E716404D02B0EE8EC8B
:1011700002F004D071503009E8EC02F012006F5018
:101180006CEC03F065EC03F070506CEC03F065EC74
:1011900003F071506CEC03F065EC03F012004FECBF
:1011A00004F05BEC03F085D8C3CF4AF0C4CF4BF01A
:1011B000260E436E4D0E426EE4EC05F0426A436A21
:1011C000446A456A466A3AC042F039BE422AB0DDF6
:1011D00015DE030E8A6F010E8B6F8C6B030E63ECB2
:1011E00003F0D6DD000EF86E380EF76E180EF66EB0
:1011F00073EC03F099EF02F04FEC04F050D8C3CF3A
:1012000042F0C4CF43F01E0E4A6E000E4B6E4A50A1
:1012100042264B5043224A6A4B6A4C6A4D6A4E6AD8
:10122000640E4A6ED1DC6EEC04F0170E4B6E810E2C
:101230004A6E33DD38C030F012004FEC04F02BD88A
:10124000C3CF42F0C4CF43F0660E4A6E000E4B6E21
:101250004A5042264B5043224A6A4B6A4C6A4D6AB6
:101260004E6A640E4A6EB0DC6EEC04F04F0E4B6EAC
:10127000EC0E4A6E12DD3828326E1200C09E17D86E
:101280008E51596EC08E120014D8C3CF67F0C4CFF0
:1012900068F02E8E12001D0E0DD0190E0BD0150EFB
:1012A00009D0110E07D00D0E05D0090E03D0050E82
:1012B00001D0010EC26E640E5A6E5A2EFED7C28243
:1012C000C2B2FED7C4CF8EF0C3CF8DF01200386EFD
:1012D0006E0E3802F3CF38F0F4CF39F038BE392A29
:1012E00039501200010E525C08E1000EF86E380E03
:1012F000F76E7E0EF66E73EC03F0020E525C08E1A0
:10130000000EF86E380EF76E900EF66E73EC03F06A
:10131000030E525C08E1000EF86E380EF76EA20E56
:10132000F66E73EC03F0040E525C08E1000EF86EEA
:10133000380EF76EB40EF66E73EC03F0050E525CC9
:1013400008E1000EF86E380EF76EC60EF66E73ECFE
:1013500003F0060E525C08E1000EF86E380EF76ED0
:10136000D80EF66E73EC03F0070E525C08E1000E27
:10137000F86E380EF76EEA0EF66E73EC03F0080E98
:10138000525C08E1000EF86E380EF76EFC0EF66E39
:1013900073EC03F0090E525C08E1000EF86E390E92
:1013A000F76E0E0EF66E73EC03F00A0E525C08E157
:1013B000000EF86E390EF76E200EF66E73EC03F029
:1013C0000B0E525C08E1000EF86E390EF76E320E0D
:1013D000F66E73EC03F00C0E525C08E1000EF86E32
:1013E000390EF76E440EF66E73EC03F012002E9A6F
:1013F000376AB8EC02F02D722DB202D0010E526E97
:101400002E8C72685BEC03F0BCD01ED9010E525CCE
:1014100001E113D9020E525C01E1EAD8030E525CDD
:1014200001E1DBD8040E525C02E1F9EC17F0050E85
:10143000525C02E1010E326E060E525C02E1020EB7
:10144000326E070E525C02E1000E306E080E525CE6
:1014500002E1030E306E090E525C02E1060E306EA0
:101460000A0E525C02E1090E306E0B0E525C02E174
:101470000C0E306E0C0E525C02E10F0E306E7DD001
:10148000E3D8010E525C01E1C5D8020E525C01E1C5
:10149000BAD8030E525C02E13CD978D9040E525CF2
:1014A00001E193DA050E525C02E1030E326E060E84
:1014B000525C02E1050E326E070E525C02E1010E33
:1014C000306E080E525C02E1040E306E090E525C62
:1014D00002E1070E306E0A0E525C02E10A0E306E17
:1014E0000B0E525C02E10D0E306E0C0E525C02E1EE
:1014F000100E306E42D0A8D8010E525C01E149D8DE
:10150000020E525C09E1040E0E5C05E0040E0E6E44
:101510002E8C726801D07ED8030E525C01E12C70D3
:10152000040E525C02E13BDE14D1050E525C02E176
:10153000040E326E060E525C02E1060E326E070E8B
:10154000525C02E1020E306E080E525C02E1050EA2
:10155000306E090E525C02E1080E306E0A0E525CCB
:1015600002E10B0E306E0B0E525C02E10E0E306E7D
:101570000C0E525C02E1110E306E366A010E526E94
:101580002D928DEC02F0FDE25BEC03F02E8C726884
:1015900012002EB60BD016D82DB804D01ED825C0F8
:1015A00026F006D025D826C025F002D006D838D996
:1015B0002E762E8C72682D80120010EE1BF020EE1D
:1015C000ABF004D020EE1BF010EEABF00C0E5A6E18
:1015D000DECFE6FF5A2EFCD712001BC020F01CC045
:1015E00021F01DC022F01EC023F01FC024F0B1D096
:1015F00020C01BF021C01CF022C01DF023C01EF033
:1016000024C01FF0A6D02D742DA41200010E0E6E62
:101610002E8C1200376A0F5206E10E2A050E0E5C60
:1016200009E30E6A07D00E2A040E0E5C03E30E6A6D
:1016300010A60E2A2E8C72681200F7D82D78F0D8DA
:101640002D802E8C72681200376AB8EC02F0010E01
:10165000525C12E1050E5A6E8DEC02F00DE3A3EC24
:1016600002F05A2EF9D7B4EC02F0A3EC02F0020E0D
:10167000526E8DEC02F0FDE252501200310433EC58
:1016800000F0056E00EE13F0040E5A6E9CEF0BF0A6
:10169000310433EC00F0056E00EE17F0040E5A6EC4
:1016A000A3EC0BF0310433EC00F0056E00EE13F008
:1016B000040E5A6E315209E1136A146A156A166AE9
:1016C000176A186A196A1A6A1200A3EF0BF023EC62
:1016D00000F0056E00EE1BF0040E5A6E1200276A31
:1016E000286A296A2A6A2B6AF2DF2DD8EE52F4DFC3
:1016F0002AD8EE52020E5A6E26D80D0E0F5C03E366
:10170000050E5A6E20D82F9425BE2F84259E88D88A
:1017100012008BD82FB4258EDADF0ED8EE52DCDF24
:101720000BD8EE52020E5A6E07D80D0E0F5C03E373
:10173000050E5A6E01D81200EE50066E52D8052AD8
:101740005A2EFAD7120062D8EE6E052A5A2EFBD70F
:101750001200010E526E2D922E8C72685BEF03F018
:10176000056A0A0E5A6E00EE09F006D8220E056EC2
:101770000A0E5A6E00EEB7F049D8EE6E052A5A2EC0
:10178000FBD7FE0E056E42D82C6E1200056A0A0EBB
:101790005A6E00EE09F006D8220E056E0A0E5A6E39
:1017A00000EEB7F0EECF06F01CD8052A5A2EFAD775
:1017B000FE0E056E2CC006F014D81200000EF86E56
:1017C0007F0EF76E000EF66EF29E2F885A6A056A3B
:1017D0000900F550066E05D8052A5A2EF9D700EFF4
:1017E00000F0A6B2FED70550A96E0650A86EA69EC0
:1017F000A69CA684F29EF2BEFDD7550EA76EAA0E39
:10180000A76EA6822FA8F28EA6941200A6B2FED7CB
:101810000550A96EA69EA69CA680A850066E120032
:1018200025502DB82650326E12002DB831C026F04A
:101830002DA831C025F01200115214E0010E115CE8
:1018400010E0020E115C0DE0030E115C2FE0040E9F
:10185000115C2FE0050E115C2FE0060E115C2FE0ED
:10186000120012000BD8440E926FBB0E916F0AD873
:10187000470E926FAE0E916F42EF0CF0200E926FFA
:10188000000E916F8290925104D8915102D88280BB
:101890001200386E080E5A6E3836D8A08294D8B02E
:1018A0008284829282825A2EF7D71200240E386EDA
:1018B00008D02C0E386E05D0A40E386E02D0040E5F
:1018C000386E829282908294829A010E906F0AD82A
:1018D000906B08D8906B06D838C090F003D88280FF
:1018E00082901200080E5A6E9037D8B0828482829D
:1018F000829282945A2EF8D712005EC093F05FC095
:1019000094F060C095F061C096F0115211E0010EA4
:10191000115C29E0020E115C23E045D0120062C088
:1019200093F063C094F064C095F065C096F0EDD775
:10193000A5DF93C091F094C092F0929F928DA2DFA8
:10194000933794379537963793379437953796373B
:1019500095C091F096C092F0929F928D42EF0CF05C
:101960003B6A3B8001D03B6A93C03AF00FD894C0E9
:101970003AF00CD895C03AF009D896C03AF006D89B
:101980003BC03AF003D8828082901200080E5A6E53
:101990003A32D8A002D0828401D08294828282928C
:1019A0005A2EF6D71200040E906F9CDF96C090F06E
:1019B00099DF95C090F096DF94C090F093DF93C0CC
:1019C00090F090DF82808290120083845BEC03F0C1
:1019D0008DEC02F0FDE2376A010E976F2BD837BE0F
:1019E0000AD037507C0B14E0972B1B0E975D02E159
:1019F000010E976F0BD037C05DF05D6C5D50FC0B36
:101A000007E09707972902E11A0E976F13D8376AF4
:101A10008DEC02F0E4E3B8EC02F0D1EC03F0010E3F
:101A2000365C03E176D900EF00F0040E365CF0E19D
:101A3000BDEF0AF0000EF86E340EF76E260EF66E4D
:101A400073EC03F0E86A63EC03F0010E975D0DE1BF
:101A5000000EF86E340EF76E380EF66E76EC03F06C
:101A600010A054D910B04FD91200020E975D0DE1AD
:101A7000000EF86E340EF76E480EF66E76EC03F03C
:101A800010A444D910B43FD91200030E975D0DE1A4
:101A9000000EF86E340EF76E580EF66E76EC03F00C
:101AA00010A234D910B22FD91200040E975D0DE1A7
:101AB000000EF86E340EF76E680EF66E76EC03F0DC
:101AC00010A624D910B61FD91200050E975D0DE19E
:101AD000000EF86E340EF76E780EF66E76EC03F0AC
:101AE00010A814D910B80FD91200060E975D0DE199
:101AF000000EF86E340EF76E880EF66E76EC03F07C
:101B000010AA04D910BAFFD81200070E975D0DE194
:101B1000000EF86E340EF76E980EF66E76EC03F04B
:101B20002FA4F4D82FB4EFD81200080E975D0DE162
:101B3000000EF86E340EF76EA80EF66E76EC03F01B
:101B400010ACE4D810BCDFD81200090E975D0DE18F
:101B5000000EF86E340EF76EB80EF66E76EC03F0EB
:101B600010AED4D810BECFD812000A0E975D09E18E
:101B7000000EF86E340EF76EC80EF66E76EC03F0BB
:101B800012000B0E975D09E1000EF86E340EF76E31
:101B9000DA0EF66E76EC03F012000C0E975D09E19A
:101BA000000EF86E340EF76EEC0EF66E76EC03F067
:101BB00012000D0E975D09E1000EF86E340EF76EFF
:101BC000FE0EF66E76EC03F012000E0E975D09E144
:101BD000000EF86E350EF76E100EF66E76EC03F012
:101BE00012000F0E975D09E1000EF86E350EF76ECC
:101BF000220EF66E76EC03F01200100E975D09E1EE
:101C0000000EF86E350EF76E340EF66E76EC03F0BD
:101C10001200110E975D0AE1000EF86E350EF76E98
:101C2000460EF66E76EC03F015EF14F0120E975D8B
:101C300009E1000EF86E350EF76E560EF66E76EC74
:101C400003F01200130E975D09E1000EF86E350ED9
:101C5000F76E680EF66E76EC03F01200140E975DC8
:101C600009E1000EF86E350EF76E7A0EF66E76EC20
:101C700003F01200150E975D09E1000EF86E350EA7
:101C8000F76E8C0EF66E76EC03F01200160E975D72
:101C900009E1000EF86E350EF76E9E0EF66E76ECCC
:101CA00003F01200170E975D09E1000EF86E350E75
:101CB000F76EB00EF66E76EC03F01200180E975D1C
:101CC00009E1000EF86E350EF76EC20EF66E76EC78
:101CD00003F01200190E975D09E1000EF86E350E43
:101CE000F76ED40EF66E76EC03F012001A0E975DC6
:101CF00009E1000EF86E350EF76EE60EF66E76EC24
:101D000003F012001200310EE8EF02F0300EE8EF9F
:101D100002F08DEC02F0FDE25BEC03F0010E975D4A
:101D200001E14AD3020E975D01E1EAD2030E975D0D
:101D300001E109D3040E975D01E1C3D2050E975D61
:101D400001E1A0D2060E975D01E157D3070E975D22
:101D500001E133D2080E975D01E175D2090E975D5E
:101D600001E152D20A0E975D01E162D10B0E975D3F
:101D700003E1010E316E50D00C0E975D03E1020EAF
:101D8000316E4AD00D0E975D03E1030E316E44D0E3
:101D90000E0E975D03E1040E316E3ED00F0E975D7F
:101DA00003E1050E316E38D0100E975D03E1060E8B
:101DB000316E32D0110E975D02E18DEF13F0120EED
:101DC000975D01E13BD3130E975D02E138EF15F00B
:101DD000140E975D02E128EF14F0150E975D02E1F5
:101DE000C3EF14F0160E975D02E173EF14F0170EB7
:101DF000975D02E1ECEF15F0180E975D02E14FEFF1
:101E000017F0190E975D02E138EF16F01A0E975D84
:101E100002E1D4EF16F0120031C025F02D98376A98
:101E200052EC0BF02F8213C09EF014C09FF015C02F
:101E3000A0F016C0A1F05BEC03F0000EF86E360EB9
:101E4000F76E580EF66E73EC03F0000E986FEAD83A
:101E5000000EF86E200EF76E200EF66E76EC03F094
:101E60009EC01BF09FC01CF0A0C01DF0A1C01EF0C2
:101E7000E8EC03F04BEC04F0E86A63EC03F09EC07E
:101E800042F09FC043F0A0C044F0A1C045F098ECE0
:101E900006F0FEEC06F00A0E8A6F060E8B6F98C0F5
:101EA0008CF0C8EC06F0375201E17ED0996B9A6B4A
:101EB0009B6B9C6B37BE3AD0985308E19E2BD8B4ED
:101EC0009F2BD8B4A02BD8B4A12B6CD0020E985D58
:101ED0000BE1640E996F99519E279A519F239B5154
:101EE000A0239C51A1235ED0040E985D0DE1100E3D
:101EF000996F270E9A6F99519E279A519F239B5154
:101F0000A0239C51A1234ED0060E985D0FE1400EF8
:101F1000996F420E9A6F0F0E9B6F99519E279A519F
:101F20009F239B51A0239C51A1233CD098530BE1AC
:101F30009E079E2907E19F079F2904E1A007A0298A
:101F400001E1A1072FD0020E985D0BE1640E996F9D
:101F500099519E5F9A519F5B9B51A05B9C51A15BE5
:101F600021D0040E985D0DE1100E996F270E9A6F27
:101F700099519E5F9A519F5B9B51A05B9C51A15BC5
:101F800011D0060E985D0EE1400E996F420E9A6FC9
:101F90000F0E9B6F99519E5F9A519F5B9B51A05B67
:101FA0009C51A15B376A5CD78DEC02F001E27BD7D4
:101FB000B8EC02F0D1EC03F0010E365C07E1982B8F
:101FC000982B080E985D01E1986B1BD0020E365CD1
:101FD00007E19807980798AF02D0060E986F08D0CF
:101FE000030E365C01E111D0040E365C01E10ED027
:101FF00019D8000EF86E200EF76E200EF66E76ECF5
:1020000003F08DEC02F0FDE22BD712009EC013F01E
:102010009FC014F0A0C015F0A1C016F03EEF0BF069
:102020004D487A00E86A63EC03F00D0E67EF03F0A9
:102030002D982F8209C09EF00AC09FF00BC0A0F01F
:102040000CC0A1F00DC0A2F05BEC03F0000EF86E26
:10205000360EF76E580EF66E73EC03F0050E986FA1
:10206000E8EC03F04BEC04F0DDDFE86A63EC03F02E
:1020700098C05AF000EE0DF0ED506CEC03F05A2EC3
:10208000FBD7375261E037BE29D0050E985D09E1D4
:10209000092AD8B40A2AD8B40B2AD8B40C2AD8B43E
:1020A0000D2A040E985D07E10A2AD8B40B2AD8B489
:1020B0000C2AD8B40D2A030E985D05E10B2AD8B47A
:1020C0000C2AD8B40D2A020E985D03E10C2AD8B46C
:1020D0000D2A010E985D01E10D2A34D0050E985DA0
:1020E0000DE1090609280AE10A060A2807E10B069C
:1020F0000B2804E10C060C2801E10D06040E985D86
:102100000AE10A060A2807E10B060B2804E10C067F
:102110000C2801E10D06030E985D07E10B060B2864
:1021200004E10C060C2801E10D06020E985D06E1A3
:102130000C060C28D8B40D06D8B40C52010E985DCC
:1021400001E10D06376A8CD78DEC02F09AE3B8EC0A
:1021500002F0D1EC03F0010E365C06E198079853CB
:1021600002E1050E986F12D0020E365C07E1982B43
:10217000060E985D02E1010E986F08D0030E365CE2
:1021800001E108D0040E365C01E10FD08DEC02F0C5
:10219000FDE266D79EC009F09FC00AF0A0C00BF018
:1021A000A1C00CF0A2C00DF01200000E056E00EEF2
:1021B00009F0050E5A6E9CEF0BF0000EF86E350E0E
:1021C000F76EFE0EF66E73EC03F0000EF86E360E30
:1021D000F76EB20EF66E73EC03F08DEC02F0FDE3D9
:1021E000D1EC03F0010E365C0EE0020E365C0BE023
:1021F000030E365C02E12F8404D0040E365C03E14A
:102200002F9489EC0BF01200000EF86E370EF76E6B
:10221000400EF66E73EC03F0BAD88DEC02F0FDE3DD
:10222000D1EC03F0010E365C0DE0020E365C0AE0E4
:10223000030E365C02E1388E04D0040E365C02E1F7
:10224000389EB4D01200000EF86E370EF76E2E0EC8
:10225000F66E73EC03F09BD88DEC02F0FDE3D1EC4D
:1022600003F0010E365C0DE0020E365C0AE0030E50
:10227000365C02E1388C04D0040E365C02E1389CF6
:1022800095D01200000EF86E360EF76E6A0EF66EDE
:1022900073EC03F07CD88DEC02F0FDE3D1EC03F09D
:1022A000010E365C0DE0020E365C0AE0030E365C71
:1022B00002E1388804D0040E365C02E1389876D00A
:1022C0001200000EF86E360EF76E460EF66E73ECC8
:1022D00003F05DD88DEC02F0FDE3D1EC03F0010ECC
:1022E000365C0DE0020E365C0AE0030E365C02E15D
:1022F000388604D0040E365C01E1389657D01200BF
:10230000000EF86E360EF76E100EF66E73EC03F0DC
:102310003ED88DEC02F0FDE3B8EC02F0D1EC03F016
:10232000010E365C0FE0020E365C0CE0030E365CEC
:1023300003E13884389205D0040E365C02E138940B
:10234000389234D01200000EF86E360EF76E220E60
:10235000F66E73EC03F01BD88DEC02F0FDE3B8ECE5
:1023600002F0D1EC03F0010E365C10E0020E365C98
:102370000DE0030E365C04E138823894838405D086
:10238000040E365C03E13892389410D01200070E28
:10239000056E06EC0CF006C038F0000EF86E350E37
:1023A000F76EFE0EF66E73EC03F0120038C006F006
:1023B000070E056EF1EF0BF0000EF86E360EF76E9D
:1023C000340EF66E73EC03F0E2DF8DEC02F0FDE309
:1023D000B8EC02F0D1EC03F0010E365C0DE0020E19
:1023E000365C0AE0030E365C02E1388004D0040E4D
:1023F000365C02E13890DAD71200000EF86E360E25
:10240000F76E7C0EF66E73EC03F0C1DF8DEC02F01C
:10241000FDE3B8EC02F0D1EC03F0010E365C0DE008
:10242000020E365C0AE0030E365C02E1388A04D004
:10243000040E365C02E1389AB9D71200000EF86E2D
:10244000360EF76E8E0EF66E73EC03F0000EF86E1D
:10245000360EF76EA00EF66E73EC03F08DEC02F004
:10246000FDE3D1EC03F0040E365C0DE0010E365CAA
:1024700006E1276A286A296A2A6A2B6A4CD18DEC00
:1024800002F0FDE2EBD78DEC02F0FDE22D98376A09
:1024900027C09EF028C09FF029C0A0F02AC0A1F05C
:1024A0002BC0A2F01B509E271C509F231D50A02321
:1024B0001E50A1231F50A2235BEC03F0000EF86E08
:1024C000360EF76E580EF66E73EC03F0000E986F32
:1024D000A9DD000EF86E200EF76E200EF66E76EC7B
:1024E00003F0E86A63EC03F09EC042F09FC043F043
:1024F000A0C044F0A1C045F0A2C046F098EC06F0A0
:10250000FEEC06F00B0E8A6F060E8B6F98C08CF0F7
:10251000C8EC06F0375201E1B8D0996B9A6B9B6B0F
:102520009C6B9D6B37BE56D098530AE19E2BD8B456
:102530009F2BD8B4A02BD8B4A12BD8B4A22BA3D056
:10254000020E985D0DE1640E996F99519E279A5184
:102550009F239B51A0239C51A1239D51A22393D043
:10256000040E985D0FE1100E996F270E9A6F995126
:102570009E279A519F239B51A0239C51A1239D519B
:10258000A22381D0060E985D11E1400E996F420E94
:102590009A6F0F0E9B6F99519E279A519F239B51C3
:1025A000A0239C51A1239D51A2236DD0080E985DBC
:1025B00011E1E10E9A6FF50E9B6F050E9C6F99511C
:1025C0009E279A519F239B51A0239C51A1239D514B
:1025D000A22359D098530EE19E079E290AE19F0736
:1025E0009F2907E1A007A02904E1A107A12901E192
:1025F000A20749D0020E985D0DE1640E996F9951C2
:102600009E5F9A519F5B9B51A05B9C51A15B9D512A
:10261000A25B39D0040E985D0FE1100E996F270E62
:102620009A6F99519E5F9A519F5B9B51A05B9C5101
:10263000A15B9D51A25B27D0060E985D11E1400E73
:10264000996F420E9A6F0F0E9B6F99519E5F9A5130
:102650009F5B9B51A05B9C51A15B9D51A25B13D0E2
:10266000080E985D10E1E10E9A6FF50E9B6F050E56
:102670009C6F99519E5F9A519F5B9B51A05B9C51AF
:10268000A15B9D51A25B376A2CD78DEC02F001E271
:1026900041D7B8EC02F0D1EC03F0010E365C07E153
:1026A000982B982B0A0E985D01E1986B1BD0020EB7
:1026B000365C07E19807980798AF02D0080E986F2C
:1026C00008D0030E365C01E111D0040E365C01E146
:1026D0000ED0A8DC000EF86E200EF76E200EF66EFF
:1026E00076EC03F08DEC02F0FDE2FBD612001B50FD
:1026F0009E5F1C509F5B1D50A05B1E50A15B1F5036
:10270000A25B9EC027F09FC028F0A0C029F0A1C006
:102710002AF0A2C02BF089EF0BF08DEC02F0FDE265
:10272000000EF86E360EF76E580EF66E73EC03F070
:102730002AD88DEC02F0FDE28DEC02F0FDE3B8EC5E
:1027400002F0D1EC03F0010E365C06E1112A070E0F
:10275000115C01E1116AE1D7020E365C06E1110657
:10276000112802E1060E116ED8D7030E365C01E186
:1027700009D0040E365C06E1080E056E11C006F0A5
:10278000F1EF0BF01200115209E1000EF86E330E5A
:10279000F76EB60EF66E73EC03F047D0010E115CC7
:1027A00009E1000EF86E330EF76EC60EF66E73EC8E
:1027B00003F03BD0020E115C09E1000EF86E330EFF
:1027C000F76ED60EF66E73EC03F02FD0030E115C8D
:1027D00009E1000EF86E330EF76EE60EF66E73EC3E
:1027E00003F023D0040E115C09E1000EF86E330EE5
:1027F000F76EF60EF66E73EC03F017D0050E115C53
:1028000009E1000EF86E340EF76E060EF66E73ECEC
:1028100003F00BD0060E115C08E1000EF86E340ECA
:10282000F76E160EF66E73EC03F0426A436A446A62
:10283000456A466A11C042F098EC06F0FEEC06F0DC
:10284000020E8A6F000E8B6F000E8C6FC8EF06F0C1
:10285000376A000EF86E360EF76EC40EF66E73EC25
:1028600003F0000EF86E370EF76ED60EF66E73ECB0
:1028700003F04FEC04F0C0C042F098EC06F0FEEC20
:1028800006F0030E8A6F000E8B6F000E8C6FC8EC83
:1028900006F065EC03F0E4EC17F0D8EC18F009EC66
:1028A00019F08DEC02F00BE3B8EC02F0D1EC03F080
:1028B000040E365C01E11200010E365C11E0375265
:1028C000F0E037BE05D037A8ECD7C02B376AC9D7A0
:1028D000376C37A803D0C007376AC3D7376CE1D746
:1028E000C6EC0BF01200000EF86E360EF76EC40E3A
:1028F000F66E73EC03F0000EF86E370EF76EC80E2E
:10290000F66E73EC03F04FEC04F012C042F0050ECB
:102910004A6EE4EC05F06EEC04F098EC06F0FEEC88
:1029200006F0040E8A6F000E8B6F000E8C6FC8ECE1
:1029300006F0000EF86E370EF76ED20EF66E76ECDD
:1029400003F08DEC02F00BE3B8EC02F0D1EC03F0F5
:10295000040E365C01E11200010E365C11E03752C4
:10296000F0E037BE05D037A8ECD7122A376AC3D7B4
:10297000376C37A803D01206376ABDD7376CE1D75A
:10298000C6EC0BF01200000EF86E360EF76EC40E99
:10299000F66E73EC03F02D84BDEC03F0000EF86EC0
:1029A000370EF76E520EF66E73EC03F0436A446A0C
:1029B000456A466ABFC042F098EC06F038506CECAD
:1029C00003F0300EE8EC02F0000EF86E370EF76EF2
:1029D000580EF66E76EC03F08DEC02F00BE3B8ECDB
:1029E00002F0D1EC03F0040E365C01E11200010E9E
:1029F000365C11E03752F0E037BE05D037A8ECD78F
:102A0000BF2B376AC8D7376C37A803D0BF07376AE0
:102A1000C2D7376CE1D7C6EC0BF01200000E63ECA6
:102A200003F0BA516CEC03F0B9516CEC03F0B851FF
:102A30006CEC03F0B7516CEC03F065EC03F0400E66
:102A400063EC03F0BE516CEC03F0BD516CEC03F091
:102A5000BC516CEC03F0BB516CEC03F065EC03F083
:102A600097EF02F08E516CEC03F08D516CEF03F098
:102A7000000EF86E360EF76EC40EF66E73EC03F0B1
:102A8000000EF86E360EF76ED60EF66E73EC03F08F
:102A90004DEC09F0E7DFA1EC02F08DEC02F0F0E381
:102AA000B8EC02F0D1EC03F0040E365C01E1120048
:102AB000010E365C01E0E4D78DEC02F0FDE28DC042
:102AC00000F18EC001F1000EF86E360EF76EDE0ECC
:102AD000F66E73EC03F04DEC09F0C4DFA1EC02F0EC
:102AE0008DEC02F0F0E3B8EC02F0D1EC03F0040E50
:102AF000365C01E11200010E365C01E0E4D78DEC9A
:102B000002F0FDE28DC002F18EC003F14FEC04F043
:102B100000C142F001C143F002C14AF003C14BF0D1
:102B200042504A5E43504B5A44504C5A45504D5ABD
:102B300046504E5A51EC04F0A00E426EF00E436E19
:102B4000190E446E4DEC06F038C0B7F039C0B8F03D
:102B50003AC0B9F03BC0BAF04FEC04F000C142F00B
:102B600001C143F0B7C04AF0B8C04BF0B9C04CF057
:102B7000BAC04DF0E4EC05F0381E391E3A1E3B1E7B
:102B80003C1E382AD8B4392AD8B43A2AD8B43B2AB9
:102B9000D8B43C2A38C0BBF039C0BCF03AC0BDF054
:102BA0003BC0BEF0000EF86E360EF76EE60EF66E07
:102BB00073EC03F08DEC02F0FDE3D1EC03F0040EB6
:102BC000365C01E11200010E365C01E0F3D75BECEC
:102BD00003F024DFC6EF0BF0000EF86E360EF76E32
:102BE000F80EF66E73EC03F0000EF86E360EF76E0C
:102BF000C40EF66E73EC03F08DEC02F0FDE3B8EC5E
:102C000002F0D1EC03F0040E365C01E11200D1ECCD
:102C100003F0010E365C01E0DFD75BEC03F0000E41
:102C2000F86E360EF76EF80EF66E73EC03F0F29E49
:102C30002F885C6A056A400E63EC03F005506CEC6B
:102C400003F006EC0CF078EC02F0A5EC02F0052A9B
:102C50005C2EF1D7000EF86E370EF76E0A0EF66E88
:102C600073EC03F097EC02F08DEC02F0FDE2120041
:102C7000000EF86E370EF76E5C0EF66E73EC03F016
:102C8000000EF86E360EF76EC40EF66E73EC03F09F
:102C90008DEC02F0FDE3B8EC02F0D1EC03F0040E91
:102CA000365C01E11200D1EC03F0010E365C01E06C
:102CB000DFD78DEC02F0FDE2000EF86E370EF76EF6
:102CC0006E0EF66E73EC03F0000EF86E370EF76EB4
:102CD000800EF66E73EC03F08DEC02F0FDE3B8ECC1
:102CE00002F0D1EC03F0010E365C15E0D1EC03F0FC
:102CF000020E365C17E0D1EC03F0030E365C19E0EF
:102D0000D1EC03F0040E365C000EF86E7E0EF76E0A
:102D1000000EF66E14D0000EF86E7B0EF76E000EED
:102D2000F66E0DD0000EF86E7C0EF76E000EF66E8D
:102D300006D0000EF86E7D0EF76E000EF66EF29E57
:102D40002F885C6A056A03EE00F006EC0CF0EE6E6C
:102D5000052A5C2EFAD703EE00F00ED8000EF86EAE
:102D6000370EF76E0A0EF66E73EC03F09AEC02F073
:102D70008DEC02F0FDE21200200EF36EF80EF61656
:102D8000080EEECFF5FF0C000900E82EFAD70A0076
:102D9000840EA66E550EA76EAA0EA76EA682000020
:102DA0000900F32EEBD712008384000EF86E370E65
:102DB000F76EA40EF66E73EC03F0000EF86E360E8E
:102DC000F76EC40EF66E73EC03F08DEC02F0FDE2CC
:102DD0008DEC02F0FDE3B8EC02F0D1EC03F0040E50
:102DE000365C01E11200D1EC03F0010E365C01E02B
:102DF000DBD78DEC02F0FDE2000EF86E370EF76EB9
:102E00006E0EF66E73EC03F0000EF86E370EF76E72
:102E1000800EF66E73EC03F08DEC02F0FDE3B8EC7F
:102E200002F0D1EC03F0010E365C15E0D1EC03F0BA
:102E3000020E365C17E0D1EC03F0030E365C19E0AD
:102E4000D1EC03F0040E365C000EF86E7E0EF76EC9
:102E5000000EF66E14D0000EF86E7B0EF76E000EAC
:102E6000F66E0DD0000EF86E7C0EF76E000EF66E4C
:102E700006D0000EF86E7D0EF76E000EF66EE4ECD6
:102E80000BF0000EF86E370EF76E0A0EF66E73EC4E
:102E900003F09AEC02F08DEC02F0FDE21200000E5D
:102EA000F86E370EF76E1C0EF66E73EC03F0000E24
:102EB000F86E360EF76EC40EF66E73EC03F08DEC02
:102EC00002F0FDE3B8EC02F0D1EC03F0040E365C46
:102ED00001E11200D1EC03F0010E365C01E0DFD716
:102EE0005BEC03F0000EF86E370EF76E1C0EF66EFC
:102EF00073EC03F0F29E2F885D6A056A03EE00F022
:102F0000400E63EC03F005506CEC03F065EC03F04D
:102F100074EC02F0EE6E066E6CEC03F0052A5D2E8A
:102F2000EFD7650E065C16E05BEC03F0000EF86E62
:102F3000380EF76E5E0EF66E73EC03F006506CEC16
:102F400003F0000EF86E380EF76E6C0EF66E73EC32
:102F500003F015D0F29E2F885D6A056A03EE00F03B
:102F6000EECF06F0F1EC0BF0052A5D2EF9D7000E3E
:102F7000F86E370EF76E0A0EF66E73EC03F097ECF0
:102F800002F08DEC02F0FDE212001D0EAF6EAC946B
:102F9000AC8AAB88AB8E1200C3C0E1FFC4C0E2FFB5
:102FA000C151E15C02E1D89012002E98E650C56F45
:102FB000F10EE15C02E115EE00F0E1CFC3F0E2CFEB
:102FC000C4F0C551D8801200080E5B6E696A6A6A47
:102FD0006B6A6C6A55EC09F08D5169268E516A2234
:102FE00053EC09F08D516B268E516C225B2EF2D77B
:102FF00012008DEC02F0FDE24DEC04F08380838240
:103000005BEC03F04FEC04F0DFDF6A506C5C02E134
:1030100069506B5C05E3270E436E0F0E426E3FD086
:1030200069C042F06AC043F0446A456A466A6B5020
:1030300042266C504322000E4B6E640E4A6E4C6A60
:103040004D6A4E6A4F6A506AE4EC05F038C042F0AF
:1030500039C043F03AC044F03BC045F03CC046F0B4
:1030600038C079F039C07AF069C04AF06AC04BF0D4
:103070004C6A4D6A4E6A6B504A5E6C504B5A4DEC2E
:1030800006F038C042F039C043F03AC044F03BC0CB
:1030900045F03CC046F038C0A3F039C0A4F098EC2D
:1030A00006F0FEEC06F0040E8A6F020E8B6F8C6B3E
:1030B000000EF86E350EF76EF80EF66E73EC03F038
:1030C000C8EC06F0A5EC02F073D865EC03F0A1D8CB
:1030D0004FEC04F0A3C042F0A4C043F0640E4A6E6B
:1030E0004A50425E4B50435A4C50445A4D50455AF8
:1030F0004E50465A5AEC04F0640E4A6EE4EC05F069
:103100006EEC04F05AEC04F0710E4A6E020E4B6E37
:103110004DEC06F06EEC04F05AEC04F0020E4A6E30
:103120004DEC06F0100E385C05E3100EA56FA66B93
:10313000A76B0BD038C0A5F042C0A6F0100E426EAF
:10314000A551425CA76FA667A707400E63EC03F08A
:10315000A567C5EC18F0A667CDEC18F0A767D0EC12
:1031600018F08DEC02F002E281B24CD7B8EC02F01C
:103170002D94839283904BEC04F081A2FED78DECCA
:1031800002F0FBE2A1EC02F01200A5C05AF0010E21
:10319000E8EC02F05A2EFBD71200000EE8EF02F026
:1031A000A7C05AF0060EE8EC02F05A2EFBD7120028
:1031B0004FEC04F069C042F06AC043F0040E4B6E5D
:1031C000E20E4A6EE4EC05F050EC04F06EEC04F014
:1031D000080E4A6E4DEC06F039C042F03AC043F09A
:1031E0003BC044F03CC045F0C0C04AF0E4EC05F000
:1031F0006EEC04F079EC04F0E4EC05F050EC04F033
:103200006EEC04F0C30E4B6E500E4A6E4DEC06F0A1
:1032100012006EEC04F0080E8A6F830E8C6F4D6AFC
:103220004E6A0F0E4C6E420E4B6E3F0E4A6E4E5063
:10323000465C0BE14D50455C08E14C50445C05E1B7
:103240004B50435C02E14A50425C04E2820E8C6FB8
:10325000060E8A6F4D6A4E6A010E4C6E860E4B6EDC
:103260009F0E4A6E4E50465C0BE14D50455C08E1A6
:103270004C50445C05E14B50435C02E14A50425CD7
:1032800004E2810E8C6F050E8A6F98EC06F0FEEC5E
:1032900006F0030E8B6FC8EC06F0570EE8EC02F058
:1032A000120010AC1200800E78EC02F00F5078EF94
:1032B00002F010AC1200810E78EC02F0315078EF81
:1032C00002F0006ED8CF01F0E0CF02F0EACF04F0B8
:1032D000E9CF03F0C2C0EAFFC1C0E9FF9EAA0ED049
:1032E000AE50ABA204D0AE50AB98AB88F7D7EE6E21
:1032F000F10EE95C02E105EE00F0F0D7EACFC2F092
:10330000E9CFC1F0F2A407D0F29466C0D6FF2DB485
:1033100080782DA48098F2A210D0D02BF1AC06D0EA
:1033200081B602D0370607D0372A05D081A602D051
:10333000370601D0372AF17CF2929EA00BD09E90E6
:10334000536653065466540657665706000ECE6EF3
:10335000A60ECF6EA1B8A1989EA204D09E925652FE
:1033600001E0560604C0EAFF03C0E9FF02C0E0FF27
:10337000005001C0D8FF1000006ED8CF01F0E0CFA0
:1033800002F002C0E0FF005001C0D8FF100000565C
:10339000312E313420202031382E31322E3132007E
:1033A00040286329444C344A414C2056612E323324
:1033B00020000C2E0000004144393833332F4144A3
:1033C000393833342000004144393835302F353115
:1033D0002020202020000041443938353120504C35
:1033E0004C2A362020000041443939353120504CD8
:1033F0004C2A342020000041443939353120504CCA
:103400004C2A352020000041443939353120504CB8
:103410004C2A3230200000414439393531206F2E9A
:1034200020504C4C20004053455420202020202088
:103430004162627275636800303120532D4D6574AE
:1034400065722020202020003032204C696368748F
:10345000206175746F2020003033204C69636874DC
:10346000207065726D2E200030342046727120313C
:10347000487A2020202020003035204B6579657265
:1034800020202020202020003036205458205A466A
:10349000207065726D2E200030372056464F3D5209
:1034A000582D5A462020200030382042616E642F6B
:1034B0004D6F64652020200030392056464F783407
:1034C00020492F516D6978003130204444532D43F9
:1034D0006F6E73742020202000003131205A462066
:1034E0004357202020202020202000003132205A65
:1034F00046204357205265766572732000003133B1
:10350000205A46204C53422020202020202000001A
:103510003134205A4620555342202020202020209C
:1035200000003135205A46204449472020202020E1
:10353000202000003136205A4620464D20202020F1
:10354000202020200000313720444453205479703B
:103550006520202000003138204C434473686966A0
:1035600074202B20525800003139204B616C2E20E2
:1035700020532D4D6574657200003230204B616C14
:103580002E204C65697374756E6700003231204DD2
:103590006974686F6572746F6E202020000032328B
:1035A0002054582068616E672074696D65200000A2
:1035B000323320456570722E205049432D3E5043D2
:1035C0000000323420456570722E2050432D3E504D
:1035D0004943000032352045657072202D3E20465B
:1035E0006C6173680000323620466C617368202D70
:1035F0003E20456570720000005357563D0040580C
:103600002020205820202065696E202061757300DD
:10361000004C696368746175746F6D6174696B20C7
:103620002000004C69636874202020202020202086
:103630002020200000532D4D65746572202020202D
:10364000202020202000003120487A204175666C1F
:103650006F6573756E672000403C2020203E20205F
:10366000202058202020206F6B00004B6579657268
:10367000202020202020202020202000005458201E
:103680005A46207065726D616E656E74200000444C
:103690006973706C617973686966743D30202000CD
:1036A000406A6120202020202020207765697465F1
:1036B00072000056464F203D205258667271202DF0
:1036C000205A4600404F4B202020202020204162DD
:1036D000627275636800005330203D200000005383
:1036E00039203D2000000053706569636865726E83
:1036F0003F2020202020200000504943202D2D2D48
:103700003E20504320205458200040466572746982
:10371000672120202020202020202000005043204E
:103720002D2D2D3E2050494320205258200000428C
:10373000616E642F4D6F646520616B746976200043
:103740000056464F783420492F51204D69786572D4
:103750002000004D543D200020487A00004565704F
:10376000726F6D202D2D3E20466C617368000053F2
:1037700070656963686572706C61747A20202000DE
:1037800040312020202032202020203320202020E3
:103790003400402020202020202020202020202015
:1037A0002020200000466C617368202D2D3E2045AE
:1037B0006570726F6D0000456570722E617566668A
:1037C0007269736368656E0000545868616E673D86
:1037D0002000206D53000066616B3D000D4D487A5E
:1037E00000000D43572000000D43577200000D4CA0
:1037F000534200000D55534200000D44494700005C
:103800000D464D2000004042616E64776563687329
:10381000656C2020202020000820566F6C7400006A
:103820004057704D3A20000000446174656E206975
:103830006D2042756666657220000055726C616489
:10384000756E672020202020202020000055726CFB
:103850006164756E67206265656E64657400004121
:103860006262727563682021212100004046616C0C
:10387000736368657320466F726D61742100403117
:1038800020412F42205354455020524954202000BB
:10389000403220413D42204D746F6E203130306BFC
:1038A0002000403320423D4120204D656D20534192
:1038B000757420004034205357562020534554201F
:1038C00055626174200040352020435720204C531E
:1038D000422055534220200040362043577220207A
:1038E0004449472020464D2020004037204D657335
:1038F00073203136306D2038306D20004038202064
:103900002036306D2034306D2033306D200040394A
:1039100020202032306D2031376D2031356D200070
:10392000403130202031326D2031306D2020366D15
:1039300020004031312020326D20207472312074FB
:10394000723220004031322020747233207472347D
:0639500020747235200016
:107F00001771C7BC0A010252060120A1070020A177
:107F1000070040420F0060E3160080841E0080844A
:107F20001E00180C00002887F9FF44018096980075
:107F3000809698000000509E1B00903A1C000103A0
:107F400040523600207538000103205C5100205C4F
:107F500051000103F0446B0060566C000103201DCA
:107F60009A00201D9A000104E089D600C0ACD80018
:107F70000104801F1401801F14010104A059410154
:107F800030B94201010490CA7B0190CA7B0101040F
:107F90006029AC01E0D2AF0101040029FC020029F4
:107FA000FC020104E0D79908E0D799080104003FDA
:107FB000AB01003FAB010104000000000000003FE6
:107FC000AB01003FAB010104000000000000003FD6
:107FD000AB01003FAB010104000000000000003FC6
:107FE000AB01003FAB010104000000000000003FB6
:107FF000AB01003FAB01010400000000000001657F
:020000040030CA
:0E000000FF32F9E0FF79BAFFFFFFFFFFFFFFBD
:00000001FF
